:020000040000FA
:100000009228A000182009142008860087160000F6
:1000100000000000000087120800A100182021083D
:10002000860087160000000000000000871208000C
:1000300089148316FF30860083120910871600008A
:1000400000000000000087120608A200A21B1E2864
:10005000891083168601831208002830A500A601A6
:10006000A60B3028A50B302808000C13C7309F05BD
:10007000AB0DAB0D2B0D9F043230A500A50B3E2818
:100080001F150C1F412808000030AB003528013037
:10009000AB0035280230AB0035280330AB003528E3
:1000A0000430AB00352883161E088312AD001E08ED
:1000B000AC0008000310A4012416AA01A901A8019C
:1000C000AD0DAC0DA80DA90DAA0DA40B6828080054
:1000D000283084007020840A7020840A70206028F0
:1000E0000008033EA300A31980000008303EA300CF
:1000F000A31B800008002A0830382908A300230E1B
:100100000F393038012023080F39303801202808F2
:10011000A300230E0F393038012023080F3930385F
:100120000120080085018601870188018901831665
:100130003F3085008601DF308700FF30880089016D
:1001400082309F008312091581309F0038300D20C6
:100150002D2038300D202D2038300D202D2001305D
:100160000D200C300D2080300D20472053205A20C8
:100170007B2087300D204A2053205A207B20C0301E
:100180000D204D2053205A207B20C7300D205020B9
:0801900053205A207B20B32804
:02400E003A3F37
:00000001FF
